:1000000009C016C015C067C113C012C011C010C00E
:100010000FC00EC011241FBECFE9CDBF20E0A0E667
:10002000B0E001C01D92A637B207E1F79ED1DFC153
:10003000E7CFFC0180811182887F877F8083628384
:10004000438397B321E030E0A90101C0440F6A95D2
:10005000EAF7842F8095892387BB48B3C9010280C2
:1000600002C0880F991F0A94E2F7842B88BB47B31C
:10007000C901038002C0880F991F0A94E2F7842BFC
:1000800087BB88B3038002C0220F331F0A94E2F7B4
:100090002095282328BB0895FC019081338191FD90
:1000A0000BC09260908328B381E090E001C0880F7C
:1000B0003A95EAF7822B0BC09D7F908328B381E0AD
:1000C00090E001C0880F3A95EAF78095822388BBBB
:1000D0000895CF93DF93EC01888180FF13C0982FA0
:1000E0009C7039F4CE01D8DF888119828B7F8860BB
:1000F00007C083FF10C099819C3368F08460877FBC
:10010000888309C082FF02C0CE01C6DF8881877F55
:100110008B7F88831982DF91CF9108958FEF809331
:10012000750041E062E081E790E083DF44E063E056
:100130008AE690E07EDF8FE697E10197F1F700C055
:100140000000E199FECF80E090E03DD18A3A99F439
:1001500081E090E038D19091710080FB91F990930B
:10016000710082E090E02FD190916A0080FB91F9BC
:1001700090936A000CC06AEA80E090E02BD160E0C6
:1001800081E090E027D160E082E090E023D186B367
:1001900090E00090730002C0959587950A94E2F76D
:1001A0008170992721E082272091710080FB20F93E
:1001B0002093710086B390E000906C0002C095958A
:1001C00087950A94E2F78170992731E0832790910F
:1001D0006A0080FB90F990936A0020FD05C0809131
:1001E0006A0080FF3AC01DC021FB662760F981E0EC
:1001F000682760FB21F92093710081E090E0EAD04C
:1002000084E022E098B3922798BB4FEF9DEE32E056
:10021000415090403040E1F700C00000815091F71C
:10022000DECF81FB662760F991E0692760FB81F9E9
:1002300080936A0082E090E0CDD084E020E198B322
:10024000922798BB4FEF9DEE32E0415090403040F6
:10025000E1F700C00000815091F78091710081FFAB
:100260000CC028B381E090E00090740002C0880FB9
:10027000991F0A94E2F7822B88BB80916A0081FF64
:100280000CC028B381E090E000906D0002C0880FA0
:10029000991F0A94E2F7822B88BB10926F0010928C
:1002A0006E001FBC13BE83B7836083BF789412BEF9
:1002B00089B7826089BF0895BB9A98E088B389277F
:1002C00088BB2FE739EA83E0215030408040E1F7D6
:1002D00000C00000F3CF1F920F920FB60F921124AF
:1002E0002F933F938F939F93EF93FF93F894809175
:1002F000710083FF05C0809172008F5F8093720050
:1003000080916A0083FF05C080916B008F5F8093AE
:100310006B00E0917000F0E086B3E05AFF4F8083FD
:10032000809170008F5F8093700080E090E02FEFED
:10033000FC01E05AFF4F3081232301968A3091055A
:10034000B9F720937500809170008A3010F01092F8
:1003500070007894FF91EF919F918F913F912F9131
:100360000F900FBE0F901F901895D8DE81E790E098
:10037000B0DE8AE690E0ADDE2091750030E00090BE
:10038000730002C0359527950A94E2F780917100B9
:1003900020FF02C08E7F01C0816080937100209198
:1003A000750030E000906C0002C0359527950A94E6
:1003B000E2F780916A0020FF02C08E7F01C0816059
:1003C00080936A00D3CFE199FECF8EBBE09A992744
:1003D0008DB30895262FE199FECF1CBA8EBB2DBB9D
:1003E0000FB6F894E29AE19A0FBE01960895F89438
:0203F000FFCF3D
:00000001FF
